:10000000830100308A002028A00003088301AE008D
:100010000B1D1428D9308312810025088F00240875
:100020008E00051510140B1183120C1C1A281010C9
:1000300005110C1083122E088300A00E200E09005B
:1000400083010330AD00FD30AC0024308400263045
:100050002B2083017B2BA60036208000840A040815
:100060002606031900342C288312AC00AD1B3F2850
:100070002D088A002C08AC0A0319AD0A82008313EC
:0E0080002D1883172C08AC0A84000008080015
:1006CC00AA01AB010310A90CA80C031C742B26085F
:1006DC00AA0727080318270AAB070310A60DA70DB6
:1006EC002808290403190034682B8B130B133B3097
:1006FC0083168500D7308100D930831281000B110D
:10070C008B16900125088F0024088E000C10831680
:10071C000C140B178B1702308312A1006330A80046
:10072C00A9012108A600A7016623FF30A600A70097
:10073C002A08A602031CA7032B08A7029D30260734
:10074C00A400FF30031800302707A500A201A30165
:10075C00A20A0319A30A2308803AA6008B302602AA
:10076C00B83003192202031CAE2B1C3021020318D3
:10077C00C12BA10AC32B0330A10762302102031C39
:10078C00942B6230A1006330A800A9012108A600B7
:10079C00A7016623FF30A600A7002A08A602031CA7
:1007AC00A7032B08A7029D302607A400FF300318CF
:1007BC0000302707A500A201A301A20A0319A30A6E
:1007CC002308803AA6008B302602B8300319220287
:1007DC00031CE32B1D302102031CF72BFD30A1075A
:1007EC00F82BA10303302102031C912BC92B3934A4
:0207FC00FF34C8
:02400E00C43FAD
:00000001FF
